:100000000200962200000000000000000000000036
:100020000000000000000000000000021CC90000E9
:1000300000000000000000000000000000000000C0
:1000400000000000000000000000000000000000B0
:1000500000000000000064000A0000000000000032
:10008000000000000000000000000002051B00004E
:100090000000000211EA75815D1201EFE582600344
:1000A000020102782E79007AC67B057C2E7D00EC59
:1000B0004D601C88828983E493A3A882A9838A82E5
:1000C0008B83F0A3AA82AB831CBCFFE31D80E07589
:1000D00082007583007CC67D05EC4D600AE4F0A3C8
:1000E0001CBCFFF51D80F27582007583007C007DCD
:1000F00000EC4D600AE4F0A31CBCFFF51D80F21279
:10010000000312031E80FE50574D20583A202566EA
:100110002C2050574D20593A2025660D0A002564A1
:100120000D0A0041542B445649444B5944460D0A8C
:100130000041542B524649444644594B0D0A004154
:10014000542B5645520D0A0041542B424155440D43
:100150000A0041542B524649440D0A0041542B4495
:100160005649440D0A0041542B5246430D0A0041A2
:10017000542B504F57450D0A0041542B434C5353B9
:100180000D0A00436F6D6D616E643A202573005255
:100190006573706F6E73653A2025730D0A004572A2
:1001A000726F723A20496E70757420737472696E42
:1001B0006720697320746F6F2073686F7274207486
:1001C0006F2073706C69742E0A005354523A2025C4
:1001D00073200D0A00253035640D0A0030313233AA
:1001E00034353637383941424344454600000475BA
:1001F000A7007597DE7597AD75FF8075EF0675A73B
:100200001075C12075A70075A90075A900E5A93072
:10021000E7FB75A90375A903E5A930E7FB43A41122
:1002200043A60175E10175E20075E341759810750B
:100230008DE6858D8B53890F438920D28ED29943C9
:10024000A50E43A61F75820022AA82AB83ACF0FDE7
:10025000900000EAF0A3EBF0A3ECF0A3EDF075A79B
:100260002075930C75C810759400900000E0FAA3F7
:10027000E0FBA3E0FCA3E0FD900143EAF0A3EBF078
:10028000A3ECF0A3EDF090A20075F04A7404121CE8
:10029000EDAA82AB83ACF0FD9001437418F0E4A3A7
:1002A000F0A3F0A3F08A828B838CF0ED121CEDAAF0
:1002B00082AB83ACF0FDE4C39AFAE49BFB74019C2F
:1002C000E49D8A958B96D2C943944075A70022AAD3
:1002D00082AB83ACF0FD900008EAF0A3EBF0A3EC56
:1002E000F0A3EDF0900004E0C0E0A3E0C0E0A3E0E4
:1002F000C0E0A3E0C0E0900008E0C0E0A3E0C0E000
:10030000A3E0C0E0A3E0C0E07407C0E07401C0E077
:100310007480C0E0121E4EE58124F5F58122900024
:100320000C74E8F0A37403F09001F412113B9025D3
:1003300080E4F5F01202491204AF121887121CB2C1
:100340001205001211CFD2AF90000CE0FAA3E0FB2F
:100350008A828B83120DCC120E02120E26121BF112
:10036000AA82AB8390000CEAF0A3EBF0C002C003BA
:10037000741EC0E07401C0E07480C0E0121E4EE53F
:100380008124FBF581120F1BAA82AB83ACF0FD9098
:1003900005C6EAF0A3EBF0A3ECF0A3EDF0120F2AF0
:1003A000AA82AB83ACF0FD9005CAEAF0A3EBF0A300
:1003B000ECF0A3EDF0120F39AA82AB83ACF0FD9004
:1003C00005CEEAF0A3EBF0A3ECF0A3EDF09005C6A8
:1003D000E0FAA3E0FBA3E0FCA3E0FDEA4B4C8DF0C8
:1003E000C2F745F0701F9005CAE0FAA3E0FBA3E056
:1003F000FCA3E0FDEA4B4C8DF0C2F745F07006C25D
:1004000091C2928004D291D2929005C6E0FAA3E004
:10041000FBA3E0FCA3E0FD9005CAE0FEA3E0FFA380
:10042000E0F8A3E0F9900135EEF0A3EFF0A3E8F0D7
:10043000A3E9F08A828B838CF0ED12188A9005CEA6
:10044000E0FAA3E0FBA3E0FCA3E0FDE4C0E0C0E031
:100450007480C0E0743FC0E08A828B838CF0ED1220
:100460001DF8AA82E58124FCF581EA7003020348A5
:1004700090001E12113B9005CEE0FAA3E0FBA3E032
:10048000FCA3E0FDE4C0E0C0E07480C0E0743FC0C5
:10049000E08A828B838CF0ED121DF8AA82E581241C
:1004A000FCF581EA70030203481219A50203489083
:1004B000012375F08012074790013175F080120713
:1004C0004790013F75F08012074790014875F08012
:1004D00012074790015275F08012074790015C7532
:1004E000F08012074790016675F08012074790016F
:1004F0006F75F08012074790017975F08002074709
:1005000075A71075980043A60175A26075A3737551
:10051000A4FF75A5FF43F304D29A22C0E0C082C0B5
:1005200083C002C003C004C005C006C007C0D075A8
:10053000D000A28CE433FA7B00A2C2E433FC7D003D
:10054000C28CC2C275A710C29F9005D2E02401F0F0
:10055000A3E03400F09005D2E0FEA3E0FFC3EE94E8
:10056000FAEF64809480400D9005D2E4F0A3F090FF
:1005700005D4E0A3E0BA0105BB0002D28CBC0105A2
:10058000BD0002D2C2D0D0D007D006D005D004D052
:1005900003D002D083D082D0E032E5829000B6F062
:1005A00075A72010C90280FB9000B6E0F59275A7F0
:1005B0000022AAF0AB83E5829000B7F0A3EBF0A392
:1005C000EAF09000B7E0FAA3E0FBA3E0FC8A828B9C
:1005D000838CF0121F3AFD60238D82C002C003C0DD
:1005E0000412059AD004D003D0020ABA00010B907D
:1005F00000B7EAF0A3EBF0A3ECF080D19000B7EAEB
:10060000F0A3EBF0A3ECF02275A72010C80280FB4A
:1006100053C83FAA9275A7008A822275A7207A0044
:100620007B0020C82675A700758214C002C0031283
:100630001108D003D00275A7200ABA00010BBAA88E
:10064000E1BB61DE75A70075820A22C2C853C83FAC
:10065000AA9275A7008A8222AAF0AB83E582900055
:10066000BAF0A3EBF0A3EAF09000BAE0FAA3E0FB43
:10067000A3E0FCC002C003C00412061BAD82D0047C
:10068000D003D002BD0A209000BAEAF0A3EBF0A399
:10069000ECF09000BAEAF0A3EBF0A3ECF08A828BC6
:1006A000838CF0E40223898A828B838CF0ED122301
:1006B00089A3AA82AB839000BAEAF0A3EBF0A3EC83
:1006C000F080B075A720A2C8920875A70022AA835F
:1006D000E5829000BDF0A3EAF09000BDE0FAA3E04F
:1006E000FB7C007D00C3EC9AED9B50477E00BE046E
:1006F000005039C002C003C004C005C0061206C3C2
:10070000E433D006D005D004D003D00260012275B6
:1007100082FAC002C003C004C005C006121108D08E
:1007200006D005D004D003D0020E80C20CBC00B5A8
:100730000D80B222C2CC30C80B9000BFE592F0A36E
:10074000E4F080F2D2CC22AAF0AB83E5829000C123
:10075000F0A3EBF0A3EAF09000C1E0C0E0A3E0C09A
:10076000E0A3E0C0E07483C0E07401C0E07480C026
:10077000E0121E4EE58124FAF581C2A09000051218
:10078000113B9000C1E0FAA3E0FBA3E0FC8A828B5E
:10079000838CF01205B290000E75F000120658908E
:1007A000000A12113BD2A0740EC0E07400C0E0E455
:1007B000C0E0748FC0E07401C0E07480C0E0121E1D
:1007C0004EE58124FAF58122AAF0AB83E582900000
:1007D000C4F0A3EBF0A3EAF09000C7E4F0A3F0901C
:1007E00000C97401F0E4A3F09000CBE4F0A3F09012
:1007F00000C4E0FAA3E0FBA3E0FC8A828B838CF0C8
:10080000121F3AFDBD2D119000C974FFF0A3F090A6
:1008100000CB7401F0E4A3F09000CBE0FDA3E0FE78
:10082000ED2AFFEE3BF88C018F82888389F0121F3E
:100830003AFFBF00030208AEC3EF648094B0406289
:1008400074B98FF063F08095F04057C002C003C0C8
:10085000049000C7E0F8A3E0F990016FE8F0A3E985
:10086000F090000AC002C003C004C005C006C00763
:100870001220F0A882A983D007D006D005D004D0DA
:1008800003D002EF3395E0FAEF24D0FFEA34FFFA09
:100890009000C7EF28F0EA39A3F0D004D003D002CB
:1008A0008004900000220DBD00010E02082090007F
:1008B000C7E0FAA3E0FB9000C9E0FCA3E0FD9001D3
:1008C0006FEAF0A3EBF08C828D830220F0AAF0ABEC
:1008D00083E5829000D6F0A3EBF0A3EAF09000D677
:1008E000E0FAA3E0FBA3E0FC8A828B838CF0122465
:1008F000DAAA82AB839000D9E4F0A3F09000DBE4A5
:10090000F0A3F09000D6E0FCA3E0FDA3E0FE8A0790
:100910008B00C3EF9407E8648094805031C004C01A
:1009200005C006749EC0E07401C0E07480C0E0128F
:100930001E4E15811581158174CAC0E07401C0E096
:100940007480C0E0121E4EE58124FAF581228C07E6
:100950008D008E018F82888389F0121F3AF5246002
:100960002C742DB52420EFB50413E8B5050FE9B5B7
:10097000060B9000D97401F0E4A3F080099000DB2D
:100980007401F0E4A3F00FBF00CA0880C79000D93B
:10099000E0FFA3E0F84F607AC002C0039000CDE012
:1009A000F525A3E0F526A3E0F52774012525FAE453
:1009B0003526FBAF2790015474012CF0E43DA3F0E1
:1009C000A3EEF09001577403F0E4A3F08A828B83C6
:1009D0008FF0C002C003C004C005C006121E78D04C
:1009E00006D005D004D003D00274042525FAE435DE
:1009F00026FBAF278A828B838FF0E412238985251B
:100A0000828526838527F0742D122389D003D00296
:100A100080589000CDE0FFA3E0F8A3E0F9900154E6
:100A2000ECF0A3EDF0A3EEF09001577403F0E4A313
:100A3000F08F82888389F0C002C003C004C005C063
:100A400006121E78D006D005D004D003D002900044
:100A5000CDE0FFA3E0F8A3E0F974032FFFE438F83A
:100A60008F82888389F0E41223899000DBE0FFA362
:100A7000E0F84F7003020AFD9000D0E0F525A3E0F6
:100A8000F526A3E0F52774012525F528E43526F59C
:100A90002985272AEA2CFFEB3DF88E01EF24FCFF85
:100AA000E834FFF8900154EFF0A3E8F0A3E9F090E8
:100AB00001577403F0E4A3F0852882852983852AF1
:100AC000F0C002C003C004C005C006121E78D006E4
:100AD000D005D004D003D00274042525FFE43526C8
:100AE000F8A9278F82888389F0E4122389852582DB
:100AF0008526838527F0742D122389806E9000D07F
:100B0000E0F528A3E0F529A3E0F52AEA2CFFEB3D68
:100B1000F88E01EF24FCFFE834FFF8900154EFF069
:100B2000A3E8F0A3E9F09001577403F0E4A3F08583
:100B30002882852983852AF0C002C003C004C0052D
:100B4000C006121E78D006D005D004D003D0029083
:100B500000D0E0FFA3E0F8A3E0F974032FFFE4382E
:100B6000F88F82888389F0E41223899000D3E0FF14
:100B7000A3E0F8A3E0F9EA2CFCEB3DFD1CBCFF016F
:100B80001D900154ECF0A3EDF0A3EEF0900157742A
:100B900001F0E4A3F08F82888389F0121E78900020
:100BA000D3E0FAA3E0FBA3E0FC74022AFAE43BFBE7
:100BB0008A828B838CF0E4022389AAF0AB83E582DE
:100BC0009000E6F0A3EBF0A3EAF0900005122255A6
:100BD000AA82AB837C00900005C002C003C004124F
:100BE0002255AD82AE838D378E3875390090000264
:100BF000122255A882A983D004D003D002882B8961
:100C00002C752D009000E6E0F52EA3E0F52FA3E073
:100C1000F530E4F8F9F531F532E531252EF533E517
:100C200032352FF5348530358533828534838535EB
:100C3000F0121F3AF536E4B536028071853682C06F
:100C400002C003C004C000C0011224BDE582D0016F
:100C5000D000D004D003D002701085338285348355
:100C60008535F0121F3AFDBD2D388805890608B874
:100C7000000109ED252EF533EE352FF5348530359D
:100C8000E531252EFDE532352FFEAF308D828E8386
:100C90008FF0121F3AFD8533828534838535F0123B
:100CA00023890531E4B531020532020C19E8252EFD
:100CB000F8E9352FF9AD30888289838DF0E412236D
:100CC000899000CDEAF0A3EBF0A3ECF09000D0E522
:100CD00037F0A3E538F0A3E539F09000D3E52BF029
:100CE000A3E52CF0A3E52DF0852E82852F8385309A
:100CF000F0C002C003C0041208CDD004D003D0025B
:100D00009000DDE0FDA3E0FEA3E0FF8A828B838CF0
:100D1000F0C002C003C004C005C006C0071207C867
:100D2000A882A983D007D006D0058D828E838FF04C
:100D3000E8122389A3E91223899000E0E0FDA3E0F3
:100D4000FEA3E0FF8537828538838539F0C005C072
:100D500006C0071207C8A882A983D007D006D0050D
:100D60008D828E838FF0E8122389A3E91223899064
:100D700000E3E0FDA3E0FEA3E0FF852B82852C834A
:100D8000852DF0C005C006C0071207C8A882A98338
:100D9000D007D006D005D004D003D0028D828E8338
:100DA0008FF0E8122389A3E91223898A828B838C2E
:100DB000F01221858537828538838539F0122185A7
:100DC000852B82852C83852DF0022185AA83E582DF
:100DD0009000E9F0A3EAF09000E9E0C0E0A3E0C0F1
:100DE000E074D5C0E07401C0E07480C0E0745EC0FF
:100DF000E07400C0E0E4C0E0122439E58124F8F595
:100E000081229005D4E0FAA3E0FB4A70189005D443
:100E1000E0A3E090005E75F0001205B21207349076
:100E200000C80206CE221206C340012290000E75B1
:100E3000F00012065812073490000E75F0001224CC
:100E4000DAAA82AB839000B4EAF0A3EBF08A048BB9
:100E500005C3EC940CED64809480403F740E9AE4DA
:100E600064808BF063F08095F040309000DD74AECC
:100E7000F0A37400F0A3E4F09000E074B0F0A37469
:100E800000F0A3E4F09000E374B2F0A37400F0A3C8
:100E9000E4F090000E75F000020BBA22AAF0AB83CA
:100EA000E5829000EBF0A3EBF0A3EAF09000EBE01A
:100EB000FAA3E0FBA3E0FC7D007E007F007800C089
:100EC00005C006EF2AF9E83BFD8C0689828D838EEA
:100ED000F0121F3AF53AE4B53A06D006D00580364E
:100EE000D006D005853A82C002C003C004C005C048
:100EF00006C007C0001224BDE582D000D007D0068E
:100F0000D005D004D003D00260050DBD00010E0F46
:100F1000BF00AC0880A98D828E83229000AEE0FADB
:100F2000A3E0FB8A828B830224929000B0E0FAA3B4
:100F3000E0FB8A828B830224929000B2E0FAA3E065
:100F4000FB8A828B83022492AAF0AB83E582900015
:100F5000EEF0A3EBF0A3EAF09000EEE0FAA3E0FBE2
:100F6000A3E0FC8A828B838CF0121F3AFD60238DF4
:100F700082C002C003C00412249FD004D003D00258
:100F80000ABA00010B9000EEEAF0A3EBF0A3ECF03C
:100F900080D19000EEEAF0A3EBF0A3ECF022AA825D
:100FA000AB83ACF0FD9000F5EAF0A3EBF0A3ECF01E
:100FB000A3EDF0900119E4F09000F5E0FAA3E0FB56
:100FC000A3E0FCA3E0FD30E72975822DC002C00339
:100FD000C004C00512249FD005D004D003D00290D5
:100FE00000F5C3E49AF0E49BA3F0E49CA3F0E49D35
:100FF000A3F09000F1E0F53FA3E0F5407C1F7D00F9
:101000009000F3E0FEA3E0FF9000F5E0F53BA3E0E5
:10101000F53CA3E0F53DA3E0F53EC3E4953BE49544
:101020003CE4953DE46480853EF063F08095F0E417
:1010300033F8C3E49EE464808FF063F08095F0E4BD
:1010400033F94870030210F48C008D011CBCFF01C1
:101050001DE824F9F541E93400F542853F43E540B8
:10106000F5443395E0F545F546900167E543F0A377
:10107000E544F0A3E545F0A3E546F0853B82853CD9
:1010800083853DF0E53EC004C005C006C0071220C0
:1010900027AA82AB83EA24DCF582EB3401F583E4F2
:1010A00093854182854283F090015FE543F0A3E59B
:1010B00044F0A3E545F0A3E546F0853B82853C83FB
:1010C000853DF0E53E121F56AA82AB83A8F0F9D009
:1010D00007D006D005D0049000F5EAF0A3EBF0A30A
:1010E000E8F0A3E9F0EE4F70030210081EBEFF0106
:1010F0001F021008EC0424F9FAE43400FB7C008A97
:10110000828B838CF0020F48E58290011AF0438EA7
:10111000407592B87593FF85929485939575910467
:1011200090011AE0FA7B00C3EB9A500BE59130E78F
:10113000FB53917F0B80F075910022AA83E582908A
:10114000011BF0A3EAF090011BE0FAA3E0FB7C0096
:101150007D00C3EC9AED9B502B7E00BE0400501D19
:101160007582FAC002C003C004C005C0061211088F
:10117000D006D005D004D003D0020E80DE0CBC0017
:10118000D10D80CE22AA82AB83ACF0FD90011DEA86
:10119000F0A3EBF0A3ECF0A3EDF090011DE0FAA3B7
:1011A000E0FBA3E0FCA3E0FDC002C003C004C00557
:1011B0008A828B838CF0ED12252DAA82AB83ACF052
:1011C000FDE58124FCF5818A828B838CF0ED22750C
:1011D000A71075C00043A60475D2F075D3F175D47D
:1011E000FF75D5FF43F308D2C222C020C0E0C0F093
:1011F000C082C083C002C003C004C005C006C007CF
:10120000C000C001C0D075D000A28CE433FA7B00CE
:10121000A2C2E433FC7D00C28CC2C275A710C2C753
:101220009005ECE0FEA3E0FF4E700302130790056B
:10123000D8E0FEA3E0FFA3E0F8A3E0F9C374509E5A
:1012400074C39FE498E4648089F063F08095F05063
:10125000319005D8E4F0A3F0A3F0A3F09005ECE4FE
:10126000F0A3F09005DCE4F0A3F09005E0E4F0A337
:10127000F0A3F0A3F0900121F0A3E4F0A3F0A3F019
:10128000806F9005D8E0FEA3E0FFA3E0F8A3E0F9AB
:10129000C374209E744E9FE498E4648089F063F0E8
:1012A0008095F050299005DC7464F0E4A3F090057B
:1012B000E0E4F0A3F0A37496F0A37442F09001214F
:1012C000E4F0A3F0A37496F0A37442F08023900599
:1012D000DC7464F0E4A3F09005E0E4F0A3F0A37400
:1012E00096F0A37442F0900121E4F0A3F0A3F0A3E0
:1012F000F09005D8E02401F0A3E03400F0A3E0343E
:1013000000F0A3E03400F09005D6E0FEA3E0FFC3B8
:1013100074649EE464808FF063F08095F0500790D1
:1013200005D6E4F0A3F09005DCE0FEA3E0FF30E793
:10133000030213C99005D6E0FEA3E0FF8E828F83DF
:10134000C002C003C004C005122492AE82AF83A8BD
:10135000F0F99005E0E0C0E0A3E0C0E0A3E0C0E069
:10136000A3E0C0E08E828F8388F0E91225D0E5816A
:1013700024FCF581E58224FF9209B392A49005D65E
:10138000E0FEA3E0FF8E828F83122492AE82AF83B1
:10139000A8F0F9900121E0C0E0A3E0C0E0A3E0C024
:1013A000E0A3E0C0E08E828F8388F0E91225D0E5CB
:1013B0008124FCF581D005D004D003D002E582243D
:1013C000FF9209B392A20214559005D6E0FEA3E065
:1013D000FF8E828F83C002C003C004C00512249216
:1013E000AE82AF83A8F0F99005E0E0C0E0A3E0C0D2
:1013F000E0A3E0C0E0A3E0C0E08E828F8388F0E944
:101400001225D0E58224FF92A4E58124FCF5819089
:1014100005D6E0FEA3E0FF8E828F83122492AE8277
:10142000AF83A8F0F9900121E0C0E0A3E0C0E0A301
:10143000E0C0E0A3E0C0E08E828F8388F0E912254F
:10144000D0E58224FF92A2E58124FCF581D005D06D
:1014500004D003D0029005D6E02401F0A3E03400CC
:10146000F0BA0105BB0002D28CBC0105BD0002D25E
:10147000C2D0D0D001D000D007D006D005D004D043
:1014800003D002D083D082D0F0D0E0D02032C2A4EA
:10149000C2A2C2A3C2A122C2A3C2A122D2A3D2A12C
:1014A00022AA82AB83ACF0FD900129EAF0A3EBF015
:1014B000A3ECF0A3EDF0900129E0F508A3E0F50915
:1014C000A3E0F50AA3E0F50BE4C0E0C0E0C0E0C093
:1014D000E0850882850983850AF0E50B122634AE83
:1014E00082E58124FCF581EE6003021598900125C8
:1014F000E0FFA3E0F8A3E0F9A3E08F82888389F0FE
:10150000122600AA82AB83C002C0031226641224F2
:1015100092AC82AD83AFF0F89005E0ECF0A3EDF073
:10152000A3EFF0A3E8F0850882850983850AF0E53A
:101530000B122600122664AC82AD83D003D0027455
:1015400064C39CFCE49DFD8A828B83C004C00512A9
:101550002664AA82AB83D005D00490016FEAF0A381
:10156000EBF08C828D831220F0AA82AB83900195E0
:101570007464F0E4A3F08A828B831226731224929F
:10158000AA82AB83ACF0FD9005E4EAF0A3EBF0A3F4
:10159000ECF0A3EDF002164EEE700302164E850835
:1015A00082850983850AF0E50B122600122664AABB
:1015B00082AB837464C39AFAE49BFB900125E0FC40
:1015C000A3E0FDA3E0FEA3E08C828D838EF0C00239
:1015D000C003122600AC82AD83C004C0051226648D
:1015E000AE82AF83D005D004D003D00290016FEE5D
:1015F000F0A3EFF08A828B83C004C0051220F0AA0A
:1016000082AB839001957464F0E4A3F08A828B83AB
:10161000122673122492AA82AB83AEF0FFD005D0BB
:10162000049005E0EAF0A3EBF0A3EEF0A3EFF08C5A
:10163000828D83122664122492AA82AB83ACF0FDC1
:101640009005E4EAF0A3EBF0A3ECF0A3EDF0900139
:1016500025E0FAA3E0FBA3E0FCA3E08A828B838C65
:10166000F0122600AA82AB83C002C003122664AC2B
:1016700082AD83D003D002C374199CE464808DF0E2
:1016800063F08095F040399005E4E0C0E0A3E0C04D
:10169000E0A3E0C0E0A3E0C0E090666675F0667489
:1016A0003F12252DAC82AD83AEF0FFE58124FCF521
:1016B00081900121ECF0A3EDF0A3EEF0A3EFF02276
:1016C0008A828B83C002C003122664AC82AD83D0B1
:1016D00003D002C374329CE464808DF063F0809583
:1016E000F040399005E4E0C0E0A3E0C0E0A3E0C032
:1016F000E0A3E0C0E090333375F073743F12252D02
:10170000AC82AD83AEF0FFE58124FCF58190012130
:10171000ECF0A3EDF0A3EEF0A3EFF0228A828B832E
:10172000C002C003122664AC82AD83D003D002C3D2
:10173000744B9CE464808DF063F08095F0403990A8
:1017400005E4E0C0E0A3E0C0E0A3E0C0E0A3E0C0A7
:10175000E090333375F073743F12252DAC82AD8366
:10176000AEF0FFE58124FCF581900121ECF0A3EDC2
:10177000F0A3EEF0A3EFF0228A828B83122664AAF4
:1017800082AB83C374649AE464808BF063F08095C9
:10179000F040399005E4E0C0E0A3E0C0E0A3E0C081
:1017A000E0A3E0C0E090333375F073743F12252D51
:1017B000AA82AB83ACF0FDE58124FCF58190012188
:1017C000EAF0A3EBF0A3ECF0A3EDF0229005E4E047
:1017D000C0E0A3E0C0E0A3E0C0E0A3E0C0E090333D
:1017E0003375F073743F12252DAA82AB83ACF0FDE4
:1017F000E58124FCF581900121EAF0A3EBF0A3EC54
:10180000F0A3EDF022AA82AB83ACF0FD900131EAA7
:10181000F0A3EBF0A3ECF0A3EDF090012DE0FAA320
:10182000E0FBA3E0FCA3E0FD900131E0FEA3E0FFBC
:10183000A3E0F8A3E0F9C006C007C000C001C006DD
:10184000C007C000C0018A828B838CF0ED121DF8A6
:10185000AA82E58124FCF581D001D000D007D00612
:10186000EA7023C0E0C0E0C0E0C0E08E828F8388D1
:10187000F0E9122634AA82E58124FCF581EA70039E
:1018800002149702149C2202148EAA82AB83ACF03D
:10189000FD900139EAF0A3EBF0A3ECF0A3EDF0909A
:1018A0000139E0FAA3E0FBA3E0FCA3E08A828B838A
:1018B0008CF0122600E5828583F09005DEF0A3E52A
:1018C000F0F0900135E0FAA3E0FBA3E0FCA3E08A8E
:1018D000828B838CF0122600AA82AB839005DCEA0F
:1018E000F0A3EBF08A828B83122492AA82AB83ACA2
:1018F000F0FD9005EAE0FEA3E0FF8E828F83C00238
:10190000C003C004C005122492AE82AF83A8F0F9D0
:10191000D005D004D003D00290012DEEF0A3EFF05B
:10192000A3E8F0A3E9F08A828B838CF0ED1218050E
:101930009005DEE0FAA3E0FB8A828B83122492AA50
:1019400082AB83ACF0FD9005DCE0FEA3E0FF8E826D
:101950008F83C002C003C004C005122492AE82AFC0
:1019600083A8F0F9D005D004D003D002900125EE71
:10197000F0A3EFF0A3E8F0A3E9F08A828B838CF068
:10198000ED1214A19005DEE0FAA3E0FB9005E8EA71
:10199000F0A3EBF09005DCE0FAA3E0FB9005EAEAA7
:1019A000F0A3EBF0229005EC7401F0E4A3F022AA7E
:1019B00083E58290013DF0A3EAF0C2AFC28C538967
:1019C000F0438901C28C758A00758C00C28DD28C5F
:1019D0007A007B00309019108D0280F80ABA00015D
:1019E0000BBA0AF0BB00EDC28C900000E4F5F022C7
:1019F000C28C758A00758C00C28DD28C7A007B00F7
:101A0000209019108D0280F80ABA00010BBA0AF072
:101A1000BB00EDC28C900000E4F5F022C28C758A08
:101A200000758C00C28D90013FE4F0A3F0D28C9041
:101A3000013DE0FAA3E0FB7C008C057E00C3ED9A3B
:101A4000EE64808BF063F08095F0503190013FE0C0
:101A5000FDA3E0FE30900C108D0280F80DBD00F467
:101A60000E80F120900C108D0280F80DBD00F40E58
:101A700080F190013FEDF0A3EEF00C80BCC28CD25F
:101A8000AF90013FE0FAA3E0FB8B058A047B007A6C
:101A900000AF8C7E00EF3395E0F8F9EE2AFAEF3BC9
:101AA000FBE83CFCE93DFDAE8AE4FF3395E0F8F944
:101AB000EE2AFAEF3BFBE83CFCE93D8A828B838C03
:101AC000F0229000051219AFAA82AB83ACF0FD9012
:101AD0000199EAF0A3EBF0A3ECF0A3EDF090000C79
:101AE000E4F5F0C002C003C004C0051226E81227C6
:101AF000AFAE82AF83A8F0F9C006C007C000C00136
:101B000090A95075F0AB744D1227DCAE82AF83A85C
:101B1000F0F9E58124FCF5818E828F8388F0E9124B
:101B20002754AE82AF83A8F0F9D005D004D003D0FB
:101B300002C3E49AE49BE49CE464808DF063F0804B
:101B400095F050088E828F8388F0E922900000E49F
:101B5000F5F0229005F0E0FAA3E0FB9005EEE0FC42
:101B6000A3E0FD90016FEAF0A3EBF08C828D83C0BF
:101B700002C003C004C0051220F0AE82AF83D005BE
:101B8000D004D003D002900195EA2CF0EB3DA3F0F5
:101B90008E828F83122673122492AA82AB83ACF0BA
:101BA000FDE4C0E0C0E0747AC0E07444C0E08A8222
:101BB0008B838CF0ED1227DCAA82AB83ACF0FDE5C1
:101BC0008124FCF581E4C0E0C0E0747AC0E0744494
:101BD000C0E08A828B838CF0ED1227DCAA82AB8373
:101BE000ACF0FDE58124FCF5818A828B838CF0EDDD
:101BF00022121AC2AA82AB83ACF0FDC002C003C09D
:101C000004C005121B53AE82AF83A8F0F9D005D0F3
:101C100004D003D0028A828B838CF0EDC006C0070B
:101C2000C000C0011227AFAA82AB83ACF0FDC00296
:101C3000C003C004C005900FDB75F0C974401225C5
:101C40002DAA82AB83ACF0FDE58124FCF5818A826C
:101C50008B838CF0ED12118512252DAA82AB83ACFB
:101C6000F0FDE58124FCF581C002C003C004C0057D
:101C700090000075F07A74441227DCAA82AB83AC22
:101C8000F0FDE58124FCF581C002C003C004C0055D
:101C900090240075F074744912252DAA82AB83AC90
:101CA000F0FDE58124FCF5818A828B838CF0ED02C6
:101CB000260075C800438E1075CAAB75CBDD75CE96
:101CC000FF75CFFFD2ADD2CA2275A700C2CFB286B0
:101CD00032AA83E582900141F0A3EAF0900141E04D
:101CE000FAA3E0FB4A6003D2CA22C2CA22AA82AB8C
:101CF00083ACF0FD900147EAF0A3EBF0A3ECF0A376
:101D0000EDF090014BE4F0A3F0A3F0A3F0900143B9
:101D1000E0FAA3E0FBA3E0FCA3E0FD754A209001FC
:101D200047E0FFA3E0F8A3E0F9A3E0FE33920AEF57
:101D30002FFFE833F8E933F9EE33FE900147EFF077
:101D4000A3E8F0A3E9F0A3EEF090014BE0FEA3E0DE
:101D5000FFA3E0F8A3E0F9EE2EFEEF33FFE833F83F
:101D6000E933F990014BEEF0A3EFF0A3E8F0A3E91B
:101D7000F0300A1E90014BE0FFA3E0F8A3E0F9A3C6
:101D8000E0FE90014B74014FF0A3E8F0A3E9F0A34B
:101D9000EEF090014BE0FEA3E0FFA3E0F8A3E0F932
:101DA000C3EE9AEF9BE89CE99D403190014BEEC356
:101DB0009AF0EF9BA3F0E89CA3F0E99DA3F09001BB
:101DC00047E0FEA3E0FFA3E0F8A3E0F99001477429
:101DD000014EF0A3EFF0A3E8F0A3E9F0D54A0280AA
:101DE00003021D1E900147E0FAA3E0FBA3E0FCA361
:101DF000E08A828B838CF022FFA88118181229199F
:101E00001228FBE96401F58222E58290014FF090EF
:101E1000014FE0F58202249FAAF0AB83E582900196
:101E200051F0A3EBF0A3EAF0900151E0FAA3E0FB3C
:101E3000A3E0FC900150E0FD9001AFEAF0A3EBF0CD
:101E4000A3ECF09001B2EDF0901E09022E50C00CF0
:101E500085810CE50C24FBFAE50C24FBF89001AF1E
:101E6000E6F008A3E6F008A3E6F09001B2EAF090ED
:101E70001E09122E50D00C22AAF0AB83E5829001ED
:101E800059F0A3EBF0A3EAF0900159E0FAA3E0FBCC
:101E9000A3E0FC90015CEAF0A3EBF0A3ECF090016E
:101EA00057E0FDA3E0FE900154E0FFA3E0F8A3E0BB
:101EB000F9ED4E60348F82888389F0121F3AF54A1B
:101EC00060271DBDFF011E0FBF0001088A828B83A2
:101ED0008CF0E54A122389A3AA82AB83900159EAC8
:101EE000F0A3EBF0A3ECF080C8900159EAF0A3EB6B
:101EF000F0A3ECF08D078E001DBDFF011EEF4860C2
:101F00001C8A828B838CF0E4122389A3AA82AB8380
:101F1000900159EAF0A3EBF0A3ECF080D7900159BF
:101F2000EAF0A3EBF0A3ECF090015CE0FAA3E0FB95
:101F3000A3E0FC8A828B838CF02220F71430F61405
:101F40008883A88220F507E6A88375830022E280B3
:101F5000F7E49322E022AA82AB83ACF0FD90016308
:101F6000EAF0A3EBF0A3ECF0A3EDF0900163E0FA4C
:101F7000A3E0FBA3E0FCA3E0FD33E433FE6013C366
:101F8000E49AF517E49BF518E49CF519E49DF51A1D
:101F900080088A178B188C198D1AAA17AB18AC19E0
:101FA000AD1A90015FE0F517A3E0F518A3E0F5196D
:101FB000A3E0F51A33E433FF6017C3E49517F51B6C
:101FC000E49518F51CE49519F51DE4951AF51E80A5
:101FD0000C85171B85181C85191D851A1E90014339
:101FE000E51BF0A3E51CF0A3E51DF0A3E51EF08AB8
:101FF000828B838CF0EDC006C007121CEDAA82AB69
:1020000083ACF0FDD007D006EF6E6013C3E49AFEF8
:10201000E49BFFE49CF8E49D8E828F8388F0228A03
:10202000828B838CF0ED22AA82AB83ACF0FD900111
:102030006BEAF0A3EBF0A3ECF0A3EDF090016BE002
:10204000FAA3E0FBA3E0FCA3E0FD33E433FE60135E
:10205000C3E49AF50DE49BF50EE49CF50FE49DF5C1
:102060001080088A0D8B0E8C0F8D10AA0DAB0EAC54
:102070000FAD10900167E0F50DA3E0F50EA3E0F5BC
:102080000FA3E0F51030E717C3E4950DF511E495C3
:102090000EF512E4950FF513E49510F514800C85F8
:1020A0000D11850E12850F138510149001B7E511DF
:1020B000F0A3E512F0A3E513F0A3E514F08A828BF8
:1020C000838CF0EDC006123612AA82AB83ACF0FD11
:1020D000D006EE6013C3E49AFEE49BFFE49CF8E4B0
:1020E0009D8E828F8388F0228A828B838CF0ED22F2
:1020F000AA83AB828BF090016FE0A4F8A9F08AF07C
:10210000E0A429F98BF0A3E0A429F5838882222298
:10211000AA83E582900173F0A3EAF0900173E0FADC
:10212000A3E0FB4A700490000022EA24FCFAEB349E
:10213000FFFB9005F2E0FCA3E0FD900175ECF0A33D
:10214000EDF0900171E4F0A3F0900175E0FCA3E0E4
:10215000FD4C6025EAB50406EBB50502801B900135
:1021600071ECF0A3EDF08C828D83E0FCA3E0FD9098
:102170000175ECF0A3EDF080D0900175E0FAA3E0DA
:102180008A82F58322AAF0AB83E582900177F0A3DF
:10219000EBF0A3EAF0900177E0FAA3E0FBA3E08A7A
:1021A000828B83122110AA82AB83EA4B60289001B4
:1021B00071E0FCA3E0FD4C700B8A828B83A3A3E447
:1021C000F0A3F0228A828B83E0FAA3E0FB8C828D5D
:1021D00083EAF0A3EBF02290017A74C0F0A37401BB
:1021E000F09001EDE493FA740193FB90017CEAF026
:1021F000A3EBF074C04401701A90017A740124C0FA
:10220000F0E43401A3F01ABAFF011B90017CEAF05C
:10221000A3EBF090017AE0FAA3E0FB9005F2EAF07C
:10222000A3EBF090017CE0FCA3E0FDEC2AFCED3B8D
:10223000FDEC24FEFCED34FFFD8A828B83ECF0A3E1
:10224000EDF08C828D83E4F0A3F08A828B83A3A3CC
:10225000E4F0A3F022AA83E58290017EF0A3EAF0E5
:1022600090017EE0FAA3E0FBC374FB9A74FF9B50DD
:10227000049000002290017E74042AF0E43BA3F055
:102280009005F2E0FAA3E0FB4A70031221D7900513
:10229000F2E0FAA3E0FB900180EAF0A3EBF09001FA
:1022A0007EE0FAA3E0FB900180E0FCA3E0FD8C82DD
:1022B0008D83E0FEA3E0FF8E158F168C008D01E567
:1022C00015C398F515E51699F5168C828D83A3A391
:1022D000E0F8A3E0F9E515C398F8E51699F9C3E825
:1022E0009AE99B400D90018274042CF0E43DA3F028
:1022F0008023900180EEF0A3EFF0900180E0FCA33A
:10230000E0FD8C828D83E0FCA3E0FD4C7098900191
:1023100082E4F0A3F0900182E0FCA3E0FD4C605D5C
:10232000900180E0FCA3E0FD74022CFEE43DFF8EF2
:10233000828F83E0F8A3E0F948700B8E828F83EAE6
:10234000F0A3EBF08037E82CF8E93DF98C828D831F
:10235000E0FEA3E0FF88828983EEF0A3EFF08C8299
:102360008D83E8F0A3E9F088828983A3A3EAF0A330
:10237000EBF0900182740428F0E439A3F09001821C
:10238000E0FAA3E08A82F5832220F71030F6118864
:1023900083A88220F507F6A88375830022F280F7D0
:1023A000F022E582900188F0900185E0FAA3E0FB3D
:1023B000A3E0FC900188E08A828B838CF012238951
:1023C00090018574012AF0E43BA3F0A3ECF022AA6B
:1023D000F0AB83E58290018DF0A3EBF0A3EAF090DF
:1023E000018DE0FAA3E0FBA3E0FC900185EAF0A3F5
:1023F000EBF0A3ECF0900189E0FAA3E0FBA3E0FC92
:1024000090018CE0FD9001AFEAF0A3EBF0A3ECF0BB
:102410009001B2EDF09023A2122E50AA82AB8390CD
:102420000185E0FCA3E0FDA3E0FE8C828D838EF0AD
:10243000E41223898A828B8322C00C85810CE50CEF
:1024400024F8FAE50C24FBF8900185E6F008A3E6F1
:10245000F008A3E6F0E50C24F8F89001AFE6F008E8
:10246000A3E6F008A3E6F09001B2EAF09023A212EE
:102470002E50AA82AB83900185E0FCA3E0FDA3E08F
:10248000FE8C828D838EF0E41223898A828B83D026
:102490000C22AC83AB827A007900748E0227B8E5F7
:1024A00082900190F0900190E0FABA0A0810990227
:1024B00080FB75990D10990280FB8A9922E5829024
:1024C0000191F0900191E0FABA30004009EA24C687
:1024D00040047582012275820022AAF0AB83E58256
:1024E000900192F0A3EBF0A3EAF07A007B00900158
:1024F00092E0FCA3E0FDA3E0FE8C828D838EF012BF
:102500001F3AFFA3AC82AD83900192ECF0A3EDF0F3
:10251000A3EEF0EF60070ABA00DF0B80DC900192B7
:10252000ECF0A3EDF0A3EEF08A828B83221237D475
:10253000BC0003023773EF60FA30D502B2D1E583F5
:10254000B4FF03023789E582B4FF0302378925838C
:1025500040072482400B0237732483145003023750
:1025600089F582EA8DF0A4A8F0EA8EF0A428F8E4B8
:1025700035F0F9EB8DF0A428E935F0F9E433CA8F92
:10258000F0A429F9EA35F0FAEBF88EF0A429F9EA7B
:1025900035F0FAE433FBEC8DF0A429F9EA35F0FAD2
:1025A000E43BFBE88FF0A42AFAEB35F0FBE433CCF4
:1025B000FD8EF0A42AFAEB35F0FBE43CFCED8FF045
:1025C000A42BFBEC35F0FC20E7031237A1023752B5
:1025D000FFA8811818122919D2D133E6400730E735
:1025E0000B7582012220E70675820022C2D11228D3
:1025F000FBE97003F5822230D101B3E433F5822286
:10260000122754700AE582458345F0700122E430B8
:10261000D112F4700BE5F0F47006E58330E7012287
:1026200090800022700AE5F07006E58320E7012221
:10263000907FFF22FFA8811818122919D2D133E602
:10264000400730E70B7582002220E70675820122E1
:10265000C2D11228FBE97003F5822220D101B3E434
:1026600033F58222E58330E709F4F583E582F4F55A
:1026700082A322AA83E582900197F0A3EAF0900159
:1026800097E0FAA3E0FB33E433FC6009C3E49AFD6E
:10269000E49BFE80048A058B068D028E03900195D3
:1026A000E0FDA3E0FE33E433FF6009C3E49DF8E4FA
:1026B0009EF980048D008E019005C0E8F0A3E9F03A
:1026C0008A828B83C004C007123802AA82AB83D0EF
:1026D00007D004EF6C600CC3E49AFCE49BFD8C8291
:1026E0008D83228A828B8322A882A983AAF0FB8809
:1026F000F0900199E0A4FCADF089F0E0A42DFDE498
:1027000035F0FE88F0A3E0A42DFDE5F03EFEE433B5
:10271000FF89F0E0A42EFEE5F03FFF88F0A3E0A4DF
:102720002EFEE5F03FFF8AF0900199E0A42EFEE531
:10273000F03FFF8BF0E0A42FFF8AF0A3E0A42FFF6F
:1027400089F0A3E0A42FFF88F0A3E0A42F8EF08DE2
:10275000838C822212389CC3749E95824039790002
:102760001238AE30D126E9F42401F582EAF43400BF
:10277000F583EBF43400F5F0ECF43400700AE582F4
:10278000458345F0700122E430E70F22EC20E71486
:1027900089828A838BF02230D10AE4F582F583F5B1
:1027A000F074802274FFF582F583F5F0747F22FCCB
:1027B000ABF0AA83A982749EF582C2D1EC30E716F1
:1027C000D2D1E9F42401F9EAF43400FAEBF434004C
:1027D000FBECF43400FC1237A10237521237D4302C
:1027E000D502B2D1BF0009BC000302379602378977
:1027F000BC0003023773E583B4FF0BE582B4FF032B
:10280000023796023773E582B4FF03023789C39516
:10281000835007247F400B02377324801450030237
:102820003789C0E0E4CCCBCAF98D4A8E4B8F4CEF90
:1028300054F0C4F54D758306854DF0EB84F582E9BF
:10284000C4F9EAC4FAEBC4FBEC540FC47803D6FC19
:1028500018EBD6FB18EAD6FA8582F0EDA4A8F0FDB5
:102860008582F0EEA428FEE435F0F88582F0EFA42E
:1028700028FFE435F0F8E99DF9EA9EFAEB9FFBECBE
:1028800098FCAD4AAE4BAF4C30E7101582E92DF9FC
:10289000EA3EFAEB3FFBE43CFC80EDC082D5839836
:1028A000C3E933F9EA33FAEB33FBEC33FCC3E99DBC
:1028B000EA9EEB9FEC9400B3E413F9D002D0E0C49D
:1028C0004AFAD003D0E0C44BFBD004D0E0F5F0547A
:1028D0000FC44CFCD082158230F40FD3EC13FCEB08
:1028E00013FBEA13FAE913F90582E930E70A7401E8
:1028F0002AFAE43BFBE43CFC02376A7901AA82E64F
:102900008F82B5821318E6B5F00E18E6B583091864
:10291000E68A82B58202790022B4800FE5F0700A5F
:10292000E5837006E58270027F00EFB6801518B669
:10293000001018B6000B18B600060808087600222A
:1029400008080822E5829001ABF09001ABE0FA7430
:1029500064C0E07429C0E090019DE0C0E0A3E0C045
:10296000E08A82229001A4E02401F0A3E03400F088
:1029700022E5829001ACF09001ACE0FA74302AFAC2
:1029800024C6500A74072AFA300B034302208A82B5
:10299000022944E5829001ADF09001ADE0FAC45403
:1029A0000FF582C002122971D00253020F8A8202EF
:1029B000297190019FE0FAA3E0FBA3E0FCA3E0FDF6
:1029C0009001A3E0FE9001AA7420F0EE2EFEED230C
:1029D00054014206EA2AFAEB33FBEC33FCED33FDFB
:1029E0009001A6E0FFC3EE9F4007EEC39FFE4302A7
:1029F000019001AAE0149001AAF09001AAE0FF70F2
:102A0000CA90019FEAF0A3EBF0A3ECF0A3EDF090E5
:102A100001A3EEF022785AE624D075F00AA4FA78E1
:102A20005BE624D02AFA9001AEF078598603BB2DDC
:102A3000079001AEC3E49AF09001A67401F09001F2
:102A4000AEE0FAC3E464808AF063F08095F0503C15
:102A50009001AA7403F09001AAE0FBBB0A00502782
:102A60009001A6E02401F0EB14244EF8EB244EF97B
:102A70008704A604772E1A9001AEEAF0EA60089067
:102A800001AAEB04F080CF9001AEEAF09001AEE035
:102A9000FA30E712784F86037850A603784F762EE7
:102AA0009001AEEA04F09001A8E0FA600E0A9001ED
:102AB000A6E0FB9001A6EA2BF0800A3016079001F1
:102AC000A6E02401F0784E8602E4BA2D0104FA70E3
:102AD000062011033012079001A6E02401F0300F08
:102AE00003022B90301053EA600875822D1229449E
:102AF000801430110875822B122944800930120687
:102B0000758220122944784F8603BB2E0F758230C0
:102B10001229449001A7E0149001A7F09001A7E0CA
:102B2000FB149001A7F09001A6E0FCC39B400302B8
:102B30002BE075823012294480E29001A7E0FB145B
:102B40009001A7F09001A6E0FCC39B50087582207D
:102B500012294480E5784E8603BB2D0875822D121C
:102B60002944801430110875822B122944800930C1
:102B70001206758220122944784F8603BB2E617598
:102B800082301229449001A7E0149001A7F08050F0
:102B9000EA601175822D1229449001A7E01490017A
:102BA000A7F0802630111175822B1229449001A7BD
:102BB000E0149001A7F0801230120F7582201229C4
:102BC000449001A7E0149001A7F0784F8602BA2E36
:102BD0000F7582301229449001A7E0149001A7F0EC
:102BE0009001AA7401F0C2189001AAE0244EF88660
:102BF00002BA4503022CDEBA2E419001AEE0FAC3C0
:102C0000E464808AF063F08095F05012758230C0E1
:102C100002122944D0021A9001AEEAF080E190013C
:102C2000AEEAF0D2189001A8E0FA704D2016030227
:102C30002CDE75822E122944022CDE30183B9001C6
:102C4000AEE0FAEA30E72D9001A8E0FBC3E464802F
:102C50008BF063F08095F05013758230C00212291A
:102C600044D0029001A8E0149001A8F00A9001AEAF
:102C7000EAF080CF9001AEEAF03018129001A8E09F
:102C8000FAC3E464808AF063F08095F050289001E4
:102C9000AAE0244EF886028A82122944301817903E
:102CA00001AAE0244EF88602BA2E0280099001A8FB
:102CB000E0149001A8F09001A7E0149001A7F09013
:102CC00001A8E0FAC3E464808AF063F08095F040E4
:102CD0000320180A9001AAE02401F0022BE89001D9
:102CE000A8E0FAC3E464808AF063F08095F05011A4
:102CF0007582301229449001A8E0149001A8F08058
:102D0000DD300F159001A7E0FA149001A7F0EA60FA
:102D10000875822012294480EB229001A8E0FA7005
:102D20000330161174072AFA9001A7E0FB9001A75F
:102D3000C39AF0800B9001A7E0FA24FA9001A7F063
:102D40009001AAE4F0784E8602BA2B17201114786D
:102D50004E762020120D9001AA7401F09001A7E098
:102D60002401F0200F239001A7E0FAC3E464808AD5
:102D7000F063F08095F05011758220122944900183
:102D8000A7E0149001A7F080DDC2189001AAE0240A
:102D90004EF88602BA0003022E29BA452A300B02E9
:102DA00076659001A8E0FAC3E464808AF063F0805D
:102DB00095F050117582301229449001A8E01490CA
:102DC00001A8F080DDD2189001AAE0FABA0200E46E
:102DD00033FA7018EA70129001A8E0FAC3E4648034
:102DE0008AF063F08095F040033018229001AAE049
:102DF000244EF886028A821229449001AAE0FA241D
:102E0000FD501C9001A8E0149001A8F080119001E1
:102E1000AAE0FABA020930160675822E12294490E9
:102E200001AAE02401F0022D8B300F239001A7E0CE
:102E3000FAC3E464808AF063F08095F050117582E3
:102E4000201229449001A7E0149001A7F080DD2210
:102E5000AA83E5829001B3F0A3EAF09001B3E0FA0F
:102E6000A3E0FB90019DEAF0A3EBF09001A4E4F055
:102E7000A3F09001AFE0FAA3E0FBA3E0FC8A828B11
:102E8000838CF0121F3AFD9001AF74012AF0E43BED
:102E9000A3F0A3ECF0ED7003023606BD250280031B
:102EA0000235FEC20FC210C211C212C213C214C236
:102EB00015C216C20CC20DC20E9001A6E4F090011C
:102EC000A7F09001A874FFF09001AFE0FAA3E0FB37
:102ED000A3E0FC8A828B838CF0121F3AFEA3AA82A5
:102EE000AB839001AFEAF0A3EBF0A3ECF09001B557
:102EF000EEF0BE25088E82122944022E728E07BF84
:102F0000300040468E07EF24C6403F9001A8E0FF06
:102F1000BFFF27C002C003C0049001A7E075F00AFC
:102F2000A4FAEE24D09001A72AF09001A7E0D004E3
:102F3000D003D002709DD2108099EF75F00AA4FFE3
:102F4000EE24D09001A82FF080899001B5E0FEBE5C
:102F50002E159001A8E0FFBFFF028003022ED39040
:102F600001A8E4F0022ED38E07BF610040128E0745
:102F7000EF2485400B9001B574DF5EF0D20B800228
:102F8000C20B9001B5E0FEBE20028075BE23030295
:102F90003010BE2A03023015BE2B02805FBE2D0208
:102FA0008055BE4202805FBE4303023093BE44039D
:102FB000023244BE450302326ABE4603023266BE96
:102FC000470302326EBE4903023244BE4C02803BCC
:102FD000BE4E03023272BE4F0302324EBE50030297
:102FE00031B7BE53030230CABE5503023256BE5833
:102FF0000302325E0232B1D20F022ED3D211022E60
:10300000D3D212022ED3D214022ED3D215022ED333
:10301000D216022ED39001A8E0FFBFFF3B3014135D
:103020009001B2E0FF14F89001B2F09001A7E6F031
:10303000022ED3C002C003C0049001B2E024FEF807
:103040009001B2F08607088602189001A7EFF0D031
:1030500004D003D002022ED33014139001B2E0FF4B
:1030600014F89001B2F09001A8E6F0022ED3C0024D
:10307000C003C0049001B2E024FEF89001B2F086D3
:1030800007088602189001A8EFF0D004D003D00200
:10309000022ED33014129001B2E0FA14F89001B26B
:1030A000F09001B5E6F080169001B2E024FEF890B1
:1030B00001B2F08602088603189001B5EAF090018B
:1030C000B5E0F5821229440232B69001B2E024FD47
:1030D000F89001B2F086020886030886041818905A
:1030E000019FEAF0A3EBF0A3ECF08A828B838CF0D3
:1030F0001224DAAA829001A9EAF09001A8E0FBBBB1
:10310000FF059001A8EAF0200F269001A7E0FBC37D
:10311000EA9B501C9001A7EBC39AF09001A7E0FA3C
:10312000149001A7F0EA600875822012294480EB10
:1031300090019FE0FAA3E0FBA3E0FC8A828B838CE2
:10314000F0121F3AFA60399001A8E0FB149001A830
:10315000F0C3E464808BF063F08095F050228A82A3
:1031600012294490019FE0FAA3E0FBA3E0FC0ABA15
:1031700000010B90019FEAF0A3EBF0A3ECF080B00C
:10318000200F030232B69001A9E0FA9001A7E0FBFC
:10319000C3EA9B40030232B69001A7EBC39AF090BA
:1031A00001A7E0FA149001A7F0EA70030232B675A5
:1031B000822012294480E89001B2E024FDF89001B9
:1031C000B2F08602088603088604181890019FEA68
:1031D000F0A3EBF0A3ECF09001A1E0FA30E7089047
:1031E00001B57443F0801FEA546060089001B57423
:1031F00050F08012EA30E6089001B57449F080067C
:103200009001B57458F09001B5E0FAF582C0021251
:10321000294475823A1229447582301229447582F4
:1032200078122944D002BA4902800EBA50028009AD
:103230009001A0E0F58212299390019FE0F582129F
:1032400029938072D2139001A6740AF080689001CD
:10325000A67408F080609001A6740AF0805890016E
:10326000A67410F08050D20C804CD20D8048D20E43
:1032700080449001B2E024FDF89001B2F086470846
:103280008648088649181890019FE547F0A3E5484D
:10329000F0A3E549F09001A4E0FFA3E0FA8547829E
:1032A0008548838549F0EF122389A3EA1223898098
:1032B000058E82122944200C09200D06200E0302DF
:1032C000335B9001B2E024FCF89001B2F086020872
:1032D000860308860408860618181890019FEAF0ED
:1032E000A3EBF0A3ECF0A3EEF090019FE0A3E0A32A
:1032F000E0A3E08A828B838CF0EE1238F19001A873
:10330000E0FABAFF069001A87406F0300E3E900174
:10331000A2E0FA53027F9001A3EAF0E0EA2A9001CA
:10332000A3F09001A1E0FA30E70D9001A3E0FA4389
:1033300002019001A3EAF09001A3E0FA2468400A98
:103340009001A3E0FABA67005002D20D300D0612C8
:103350002D1A022E72122A15022E729001A6E0FA80
:103360007003022E729001B67453F030144790012E
:10337000B2E014F89001B2F0E6FA3395E0FBFCFEFF
:1033800090019FEAF0A3EBF0A3ECF0A3EEF0301372
:103390000302342790019FE0FAA3E0A3E0A3E07BBF
:1033A000007C007E0090019FEAF0A3EBF0A3ECF01C
:1033B000A3EEF080723015299001B2E024FCF89061
:1033C00001B2F086020886030886040886061818EB
:1033D0001890019FEAF0A3EBF0A3ECF0A3EEF080CD
:1033E000469001B2E024FEF89001B2F08602088611
:1033F0000318EB3395E0FCFE90019FEAF0A3EBF09D
:10340000A3ECF0A3EEF020131E90019FE0FAA3E0DE
:10341000FBA3E0A3E07C007E0090019FEAF0A3EB19
:10342000F0A3ECF0A3EEF030163E90019FE0FAA37B
:10343000E0FBA3E0FCA3E0FEEA4B4C4E602A9001C7
:10344000A6E0FABA0808758230122944801ABA1028
:1034500017758230122944300B087582781229447E
:10346000800675825812294430133090019FE0FA8B
:10347000A3E0FBA3E0FCA3E0FE30E71DC3E49AFA5F
:10348000E49BFBE49CFCE49EFE90019FEAF0A3EB2E
:10349000F0A3ECF0A3EEF08002C2139001A9E4F0D7
:1034A000D21778539001A3E4F0C0001229B2D000E3
:1034B0002017129001A3E0C4FAE6FB4AF618900127
:1034C000B6E8F080069001A3E0FAF69001A9E024A6
:1034D00001F0B21790019FE0FAA3E0FBA3E0FCA388
:1034E000E0FEEA4B4C4E70BC9001B6E8F09001A7AC
:1034F000E0FA70069001A77401F0201024200F213B
:103500009001A9E0FA0A9001A7E0FBC3EA9B5011E1
:103510007582201229449001A7E0149001A7F08041
:10352000DF30131175822D1229449001A7E0149009
:1035300001A7F0802D9001A9E0FA602630111175E5
:10354000822B1229449001A7E0149001A7F0801269
:1035500030120F7582201229449001A7E0149001C7
:10356000A7F0200F239001A7E0FA149001A7F09094
:1035700001A9E0FBC39A502C3010047A3080027A03
:10358000208A8212294480DD9001A7E0FA9001A9E7
:10359000E0FBC39A50099001A7EAC39BF080059015
:1035A00001A7E4F09001B6E0F89001A9E0FA1490C8
:1035B00001A9F0EA602AB21720170C08E6C4540FDC
:1035C000FA9001A3F0800A860253020F9001A3EA49
:1035D000F09001A3E0F582C000122971D00080C9EB
:1035E000200F03022E729001A7E0FA149001A7F0B9
:1035F000EA7003022E7275822012294480E88D82BF
:10360000122944022E729001A4E0FAA3E08A82F506
:103610008322AA82AB83ACF0FD9001BBEAF0A3EB5E
:10362000F0A3ECF0A3EDF09001BFE4F09001BBE05B
:10363000FAA3E0FBA3E0FCA3E0FD7E009001B7E06D
:10364000F54AA3E0F54BA3E0F54CA3E0F54D235478
:1036500001FF7074C006E54A254AFFE54B33F8E5E3
:103660004C33F9E54D33FE9001B7EFF0A3E8F0A33A
:10367000E9F0A3EEF09001B7E0F54AA3E0F54BA323
:10368000E0F54CA3E0F54DC3EA954AEB954BEC957C
:103690004CED954DD0065027E54DC313F54DE54C47
:1036A00013F54CE54B13F54BE54A13F54A9001B77A
:1036B000F0A3E54BF0A3E54CF0A3E54DF080090E37
:1036C0009001BFEEF002363C9001BFE0FA9001BBE2
:1036D000E0FBA3E0FCA3E0FDA3E0FE9001B7E0F572
:1036E0004AA3E0F54BA3E0F54CA3E0F54DC3EB9501
:1036F0004AEC954BED954CEE954D40179001BBEB88
:10370000C3954AF0EC954BA3F0ED954CA3F0EE95E4
:103710004DA3F09001B7E0FBA3E0FCA3E0FDA3E024
:10372000C313FEED13FDEC13FCEB139001B7F0A3F4
:10373000ECF0A3EDF0A3EEF08A031AEB708F90018A
:10374000BBE0FAA3E0FBA3E0FCA3E08A828B838CBE
:10375000F022B98003EA13B34010EA2401FAE43BF3
:10376000FBE43CFC50047C800582BC000EBB000BDB
:10377000BA0008E4F5F0F583F58222A2D1E58213C0
:103780008CF092F78B838A8222E4F583F58275F0C0
:1037900080F4A2D11322E4F583F58275F0C0747F22
:1037A000227804EC7011E58224F8500AF582E4C90D
:1037B000CACBFCD8EF22EC7820058220E713D58213
:1037C0000122C3E933F9EA33FAEB33FBEC33FCD8DB
:1037D000EA158222AA82AB83A2F73392D16002D289
:1037E000F7F582ACF0E58124F9F8E6FD08E6FE087D
:1037F00086F008E6A2F73392D56002D2F7F583AFE0
:10380000F022AA83E5829005C2F0A3EAF09005C4F5
:10381000E4F0A3F09005C0E0FAA3E0FB7C10900573
:10382000C2E0FDA3E0FE339219EECD25E0CD33FEDC
:103830009005C2EDF0A3EEF09005C4E0FDA3E0CD4D
:1038400025E0CD33FE9005C4EDF0A3EEF030191263
:103850009005C4E0FDA3E0FE9005C474014DF0A303
:10386000EEF09005C4E0FDA3E0FEC3ED9AEE9B40B0
:103870001D9005C4EDC39AF0EE9BA3F09005C2E045
:10388000FDA3E0FE9005C274014DF0A3EEF0DC8EC6
:103890009005C2E0FAA3E08A82F58322AA82AB8374
:1038A000A2F73392D16002D2F7F582ACF0226040E9
:1038B000F82582500274FFF582E824F8501ECCCB24
:1038C000CAF9E4CC24F85014CBCAF9E4CB24F8505C
:1038D0000BCAF9E4CA24F8500379002224086010C6
:1038E000F8C3EC13FCEB13FBEA13FAE913F9D8F174
:1038F00022C0E0F84582458345F07009F5F0FBFCF5
:10390000FDFE0239BFE823A2F792E0F8A982AA835C
:10391000D2F7ABF07C007E07C3749798404074FFE9
:103920002EFE740A89F0A4F985F082740A8AF0A444
:10393000FA85F083740A8BF0A4FB740529F9EA3543
:1039400082FAEB3583FB740035F0FCC3EC13FCEB1F
:1039500013FBEA13FAE913F908EC70EF80BAE8C335
:10396000947FF88B838EF0E4FBFCFDFEFF08C3E937
:1039700033F9EA33FAE58333F583EB3BD4FBEC3CD4
:10398000D4FCED3DD4FDEE3ED4FEEF3FD4FF602DE0
:1039900005F074052BD4FBE43CD4FCE43DD4FDE4F9
:1039A0003ED4FEE43FD4FF758204C3EF13FFEE1351
:1039B000FEED13FDEC13FCEB13FBD582EDD8AF78D5
:1039C0004ED0E020E704762B8002762D087906E7BA
:1039D000C4540F4430F608B90603762E08E7540F96
:1039E0004430F60819B902E7764508E5F020E70407
:1039F000762B8004762DF4040875F00A844430F6A2
:103A000008E5F04430F608E4F690004E75F04022E8
:00000001FF
